:0300000002435662
:03000300024BCDE0
:03000B00024BD2D3
:03001300024B920B
:03001B00024BD5C0
:03002300021B3984
:03002B000243E2AB
:03003300023FF396
:03003B00024BC0B5
:0300430002470071
:03004B00023FFC75
:030053000237FA77
:03005B00024BC78E
:030063000246FC56
:1005000012011001000000406A080101000101020F
:1005100000010902B80103010080A00904000000E5
:10052000010100000A2401000156000201020C240E
:100530000201010100060000000015240605010269
:10054000030000000000000000000000000000099F
:1005500024030204030005000C240203010200022C
:10056000000000000D240606030203000000000046
:100570000009240304010100060009040100000130
:100580000200000904010102010200000724010128
:10059000000100112402010202100344AC0080BBE0
:1005A0000000770109050A05840101008F07250174
:1005B0000100000009058F01030001060009040184
:1005C000020201020000072401010001000E2402C2
:1005D000010602100244AC0080BB0009050A054C6C
:1005E0000201008F0725010100000009058F0103AA
:1005F00000010600090401030201020000072401B2
:10060000010001000E2402010603180244AC008020
:10061000BB0009050A05720301008F0725010100CF
:10062000000009058F01030001060009040104020E
:1006300001020000072401010001000B2402010255
:1006400003180100770109050A05460201008F071A
:1006500025010100000009058F01030001060009C2
:10066000040200000102000009040201010102006D
:1006700000072401040001001124020102021003FA
:1006800044AC0080BB0000770109058C05840101A2
:100690000000072501010200000904020201010215
:1006A00000000724010400010011240201020318C4
:1006B0000344AC0080BB0000770109058C054602AD
:1006C00001000007250101020000050C0901A1013C
:1006D000050C09E9050C09EA1500250195027501CB
:1006E0008142950175068101050C0900050C090080
:1006F0001500250195027501910695017506910376
:10070000C004030904180345004D00410047004997
:10071000004300200047006D00620048001E0345B2
:10072000006D006100670069006300200045004D16
:10073000004900200032007C0036002A0343006F8D
:10074000006E006600690067007500720061007449
:100750000069006F006E0020005300740072006991
:10076000006E006700220349006E0074006500728D
:100770000066006100630065002000530074007291
:090780000069006E006700000032
:100789007400F58690FDA57C05A3E582458370F983
:01079900223D
:10079A00907FD6E04480F0438701000000000022E9
:1007AA00C0D0C0E08FE0C0E08EE0C0E08DE0C0E0E5
:1007BA008CE0C0E0C082C0830586C084C085E5188D
:1007CA00B402030207D9B401030207DE0207FA7D65
:1007DA0001020816E51914F519C3B513030207F542
:1007EA005009B400EA75190A0207D97D00020816F1
:1007FA00E51914F519C3B514030208115009B40018
:10080A00CE75190A0207D97D020208167C05907F67
:10081A0099E05440DC03020843B4001D907FE3745E
:10082A007BF0A37480F0907FE27440F0907FE5F053
:10083A00907FE27400F00208180586907FE27480C7
:10084A00F0907965E0B4010302089EB4020302083D
:10085A0096B4030302088EB40403020886B405039F
:10086A0002087EB406030208760208F40586907F21
:10087A006C0208E90586907F6C0208DD0586907F88
:10088A006C0208CF0586907F6C0208C00586907FAF
:10089A006C0208B20586907F6CF000F000F000F060
:1008AA000DEDB42DF40208F4F0F0F0F0F0F00DEDD7
:1008BA00B42DF50208F4F000F000F000F00DEDB4EC
:1008CA0031F40208F4F0F0F0F0F0F00DEDB431F587
:1008DA000208F4F0F0F0F00DEDB461F70208F4F05C
:1008EA00F0F0F0F0F00DEDB461F5907FE27400F0F5
:1008FA00D085D0840586D083D082D0E0FCD0E0FDBC
:05090A00D0E0FED0E08A
:06090F00FFD0E0D0D02271
:10091500C0D0C0E0C082C083907F6FE50CF0E50DCC
:0D092500F0E50EF0D083D082D0E0D0D022DB
:10093200C0D0C0E08FE0C0E08EE0C0E0C082C083E3
:100942000586C084C085907970E0FFBF0003020A6B
:10095200B8907F96E04480F0907FE27480F0907FC0
:1009620062E00586907FE27400F0907F96E0547F0B
:10097200F0907FE27480F0907988E0B4010302097C
:10098200BEB402030209C3B403030209ACB40403F4
:1009920002099A0586020AB2EF5403FEEF030354DA
:1009A2003FFF907F6305860209C9EF5403FEEF0300
:1009B20003543FFF907F630586020A360586020ACA
:1009C200A50586020A8EE0E0E0E0E0E00586E0E0D0
:1009D200E00586E0E0E0E0E0E00586E0E0E00586B4
:1009E200E0E0E0E0E0E00586E0E0E00586E0E0E06F
:1009F200E0E0E00586E0E0E00586DFCAEEB4000351
:100A0200020AB2B40103020A25E0E0E0E0E0E005F8
:100A120086E0E0E00586E0E0E0E0E0E00586E0E098
:100A2200E00586E0E0E0E0E0E00586E0E0E0058663
:100A3200020AB2E0E0E0E00586E0E00586E0E0E000
:0D0A4200E00586E0E00586E0E0E0E00586E6
:100A4F00E0E00586E0E0E0E00586E0E00586DFD641
:100A5F00EEB40003020AB2B40103020A80E0E0E040
:100A6F00E00586E0E00586E0E0E0E00586E0E005F1
:100A7F0086E0E0E0E00586E0E00586020AB2E0E00D
:100A8F00E0E0E0E0E0E0E0E0E0E0E0E0E0E0E0E057
:100A9F00DFEC020AB2E0E0E0E0E0E0E0E0E0E0E01E
:100AAF00E0DFF2907FE27400F0D085D0840586D02D
:0E0ABF0083D082D0E0FED0E0FFD0E0D0D02285
:100ACD00C082C083C0E0E8C0E078D1E814F870FBC4
:0A0ADD00D0E0F8D0E0D083D08222F0
:100AE700C0D0C0E08FE0C0E08EE0C0E08DE0C0E0A5
:100AF7008CE0C0E0758600C082C0830586C084C0D4
:100B0700857E0090798EE0B400167401F09006CAD5
:100B1700A3A3A3A3A3A3A3E0FF90798DF0020B39AE
:100B270090798DE0FF90798FE0FD907990E0FC025D
:100B37000B469006CA0586907F000586020B518DED
:100B4700848C850586907F000586E0A30586F0A343
:100B57000EEEB44003020B6C0586DFEE90798E74BF
:100B670000F0020B820586AD84AC8590798FEDF09D
:100B7700907990ECF090798D1FEFF0907FB5EEF0C3
:100B8700D085D0840586D083D082D0E0FCD0E0FD2C
:0B0B9700D0E0FED0E0FFD0E0D0D02284
:100BA200C0D0C0E0C082C083907FAEE054E0F0903D
:100BB2007F96E0440854FBF0907F97E054BFF0909A
:100BC2007FE3747BF0907FE47440F0907978E0905A
:100BD2007B40F0907FE27448F0907FE5E0907FE206
:100BE2007400F0907F96E054F74404F0907FE37431
:100BF2007BF0907FE47440F0907979E0907B40F054
:100C0200907FE27448F0907FE5E0907FE27400F01C
:100C1200907F96E054F3F0907FAEE0441FF0D083D3
:070C2200D082D0E0D0D02207
:100C2900C0D0C0E0C083C08290792FE064FFC324A4
:0B0C390001F0D082D083D0E0D0D022A8
:100C4400BB010689828A83E0225002E722BBFE02AE
:090C5400E32289828A83E49322E1
:100C5D00BB010CE58229F582E5833AF583E022504C
:100C6D0006E92582F8E622BBFE06E92582F8E22296
:0D0C7D00E58229F582E5833AF583E49322B0
:100C8A00BB010689828A83F0225002F722BBFE0149
:020C9A00F32243
:100C9C00F8BB010DE58229F582E5833AF583E8F08E
:100CAC00225006E92582C8F622BBFE05E92582C83A
:020CBC00F22222
:100CBE00C2D5EC30E709B2D5E4C39DFDE49CFCEE51
:100CCE0030E715B2D5E4C39FFFE49EFE120E40C37B
:100CDE00E49DFDE49CFC8003120E4030D507C3E476
:060CEE009FFFE49EFE22C0
:100CF400C5F0F8A3E028F0C5F0F8E582158270028B
:060D04001583E038F02227
:100D0A00BB0110E58229F582E5833AF583E0F5F027
:100D1A00A3E0225009E92582F886F008E622BBFE04
:100D2A000AE92582F8E2F5F008E222E5832AF5834A
:080D3A00E993F5F0A3E993220F
:100D4200E88FF0A4CC8BF0A42CFCE98EF0A42CFC50
:100D52008AF0EDA42CFCEA8EF0A4CDA8F08BF0A4CE
:100D62002DCC3825F0FDE98FF0A42CCD35F0FCEB2D
:100D72008EF0A4FEA9F0EB8FF0A4CFC5F02ECD39F2
:0F0D8200FEE43CFCEAA42DCE35F0FDE43CFC225F
:100D9100EB9FF5F0EA9E42F0E99D42F0E89C45F0B8
:010DA100222F
:100DA200BB010DE58229F582E5833AF583020EA1A6
:100DB2005007E92582F8020E95BBFE07E92582F865
:100DC200020EADE58229F582E5833AF583020EB97A
:100DD200BB010DE58229F582E5833AF583020ED542
:100DE2005007E92582F8020EC9BBFE07E92582F801
:040DF200020EE122EA
:100DF600BB010DE58229F582E5833AF583020F06EC
:100E06005007E92582F8020EEDBBFE07E92582F8B8
:040E1600020F37226E
:100E1A00D083D082F8E4937012740193700DA3A367
:100E2A0093F8740193F5828883E47374029368607B
:060E3A00EFA3A3A380DF7B
:100E4000BC000BBE0029EF8DF084FFADF022E4CC96
:100E5000F875F008EF2FFFEE33FEEC33FCEE9DEC5F
:100E6000984005FCEE9DFE0FD5F0E9E4CEFD22EDA5
:100E7000F8F5F0EE8420D21CFEADF075F008EF2FEF
:100E8000FFED33FD4007985006D5F0F222C398FDE0
:050E90000FD5F0EA227D
:0C0E9500E6FC08E6FD08E6FE08E6FF2289
:0C0EA100E0FCA3E0FDA3E0FEA3E0FF22C4
:0C0EAD00E2FC08E2FD08E2FE08E2FF2281
:100EB900E493FCA3E493FDA3E493FEA3E493FF224C
:0C0EC900ECF608EDF608EEF608EFF62255
:0C0ED500ECF0A3EDF0A3EEF0A3EFF02290
:0C0EE100ECF208EDF208EEF208EFF2224D
:100EED00D083D082E493F608740193F608740293CC
:090EFD00F608740393F674047303
:100F0600A8828583F0D083D082120F1D120F1D1286
:100F16000F1D120F1DE473E493A3C583C5F0C583AB
:100F2600C8C582C8F0A3C583C5F0C583C8C582C835
:010F36002298
:100F3700D083D082E493F208740193F20874029389
:090F4700F208740393F2740473C0
:100F5000C2AFD22C907F937430F0907F9C74BFF01E
:100F6000907F96E05430F0907F947430F0907F9DA5
:100F700074CFF0907F9774A0F0907F9574CCF0E4DC
:100F8000907F9EF0C22DC22AC22BC22E907974048B
:100F9000F0122E941249E2124BE612320D123B0D62
:100FA0001241FD123E99E51F7018751F011217FFBF
:100FB000122FFF1249C8124BD8124BDA12496F1286
:100FC0001B4012398D907FAFE04401F0907FAEE07E
:100FD000441FF0907FAC74FFF0907FADF0907FDE07
:100FE000F0907FDFF0907FABF0907FA9F0907FAA28
:100FF000F05391EF43D820D2E843D82043A8802271
:10100000907963E014604414700221D0147002419E
:10101000D914700261D7240460028156E490797873
:10102000F090797BE0907979F04401F054FDF090F4
:10103000797BF0E4907988F0A2AF33F512C2AF1259
:101040000BA2E51270028156D2AF2290792DE06496
:10105000017079907FF2F0907FF37430F0907FFF11
:1010600074FCF0E4907978F090797BE0907979F0F5
:101070004401F04402F090797BF0A2AFE433F51222
:10108000C2AF120BA29079787402F0907984E0904C
:101090007979F090797FE0B40109907979E054FE94
:1010A000F08007907979E04401F0907979E054FD7F
:1010B000F054FBF0907984F0120BA29079827404C2
:1010C000F090798814F0E5126002D2AF90792DE0AB
:1010D00064027079907FF2F0907FF37434F0907F27
:1010E000FF74FCF0E4907978F090797BE090797966
:1010F000F04401F04402F090797BF0A2AFE433F5C4
:1011000012C2AF120BA29079787402F0907984E049
:10111000907979F090797FE0B40109907979E05481
:10112000FEF08007907979E04401F0907979E0440D
:1011300002F054FBF0907984F0120BA29079827443
:1011400004F090798814F0E5126002D2AF90792D06
:10115000E0640360028156907FF2F0907FF3746444
:10116000F0907FFF74FCF0E4907978F090797BE068
:10117000907979F04401F04402F090797BF0A2AFCD
:10118000E433F512C2AF120BA29079787402F0909A
:101190007984E0907979F090797FE0B401099079D1
:1011A00079E054FEF08007907979E04401F090797D
:1011B00079E04404F0907984F0120BA29079827463
:1011C00004F090798814F0E51270028156D2AF22B3
:1011D00090792DE06401707A907FF2F0907FF37443
:1011E00088F0907FFF74FCF0E4907978F090797B40
:1011F000E0907979F04401F054FDF090797BF0A211
:10120000AFE433F512C2AF120BA29079787402F0FA
:10121000907984E0907979F090797FE0B401099039
:101220007979E054FEF08007907979E04401F090FC
:101230007979E054FDF054FBF0907984F0120BA220
:10124000907982740CF09079887401F0E512600254
:10125000D2AF90792DE0640260028156907FF2F067
:10126000907FF37494F0907FFF74FCF0E4907978B1
:10127000F090797BE0907979F04401F054FDF090A2
:10128000797BF0A2AFE433F512C2AF120BA29079D2
:10129000787402F0907984E0907979F090797FE029
:1012A000B40109907979E054FEF08007907979E0F3
:1012B0004401F0907979E04402F054FBF090798495
:1012C000F0120BA2907982740CF09079887401F07E
:1012D000E51270028156D2AF2290792DE064017040
:1012E00077907FF2F0907FF374CCF0907FFF74FCE6
:1012F000F0E4907978F090797BE0907979F054FC83
:10130000F090797BF0A2AFE433F512C2AF120BA2DA
:101310009079787402F0907984E0907979F09079FE
:101320007FE0B40109907979E054FEF0800790796C
:1013300079E04401F0907979E054FDF054FBF090AD
:101340007984F0120BA29079827412F090798874EB
:1013500002F0E5126002D2AF90792DE0640270775E
:10136000907FF2F0907FF374E0F0907FFF74FCF0D8
:10137000E4907978F090797BE0907979F054FCF002
:1013800090797BF0A2AFE433F512C2AF120BA290BA
:1013900079787402F0907984E0907979F090797F8F
:1013A000E0B40109907979E054FEF08007907979F2
:1013B000E04401F0907979E04402F054FBF0907938
:1013C00084F0120BA29079827412F09079887402E2
:1013D000F0E5126002D2AF90792DE064037077904F
:1013E0007FF2F0907FF37494F0907FFF74FCF0E450
:1013F000907978F090797BE0907979F054FEF04420
:1014000002F090797BF0A2AFE433F512C2AF120B79
:10141000A29079787402F0907984E0907979F090D4
:10142000797FE0B40109907979E054FEF08007906B
:101430007979E04401F0907979E04404F09079847E
:10144000F0120BA29079827406F09079887404F0FF
:07145000E5126002D2AF2299
:10145700C228C229907FE8E0120E1A14840014E013
:101467000114F602167C2116BE2215918015D18132
:10147700162E8216CFA11705A20000170A907FE942
:10148700E014601124FE602824FE603B24FC7040B9
:10149700124A2AE116124BE04002E116907FEAE079
:1014A700B40104C22AE116907FB4E04401F0E116CA
:1014B700124BE2907FEAE0B40104D22AE116907F52
:1014C700B4E04401F0E116907FB4E04401F0E11686
:1014D700907FB4E04401F0E116907FE9E024F570D5
:1014E7000512479CE116907FB4E04401F0E11690A5
:1014F7007FE9E024FD605424026002A188124BE0DA
:101507004002E116907FEAE07038907FECE0F454F7
:1015170080FFC4540FFFE054072F25E024B4F58261
:10152700E4347FF583E4F0907FECE05480FF1313FD
:1015370013541FFFE054072F907FD7F0E04420F0AB
:10154700E116907FB4E04401F0E116124BE240024D
:10155700E116907FEAE07020907FECE0F45480FF82
:10156700C4540FFFE054072F25E024B4F582E43478
:101577007FF5837401F0E116907FB4E04401F0E158
:1015870016907FB4E04401F0E116907FE9E0601225
:1015970024F860092402702912171EE116124BA0C5
:1015A700E116124BDEA22AE433FF25E0FFA22BE46B
:1015B700334F907F00F0E4A3F0907FB57402F0E121
:1015C70016907FB4E04401F0E116907FE9E06037C0
:1015D70024F6602E24047041907FEBE024DE600E39
:1015E700047016D229907FB4E04401F0E116D229A5
:1015F700907FB4E04401F0E116907FB4E04401F03D
:10160700E116124463E116124BDEE4907F00F0A36B
:10161700F0907FB57402F0E116202907907FB4E0BF
:101627004401F0C229E116907FE9E024F4603424F4
:101637000C7039124BDE907FECE0F45480FFC454F9
:101647000FFFE054072F25E024B4F582E4347FF53B
:1016570083E054FD907F00F0E4A3F0907FB574021F
:10166700F0E116907FB4E04401F0E116907FB4E01A
:101677004401F0E116907FE9E024F6601214601A45
:101687002402701DD228907FB4E04401F08012D26A
:1016970028907FB4E04401F08007907FB4E04401D4
:1016A700F020280F9079857401F012496F907FC55B
:1016B7007402F0C22880589079867401F012496F3D
:1016C700907FC57402F08047907FE9E024FE6012A6
:1016D70014601A2402701DD228907FB4E04401F0F0
:1016E7008012D228907FB4E04401F08007907FB445
:1016F700E04401F0202803121A7BC2288011122C23
:101707002B800C124BE45007907FB4E04401F0901B
:071717007FB4E04402F02260
:10171E00124BDC4002E1E3907FEBE024FE601E14EE
:10172E00604614606E147002E1D424046002E1DCA1
:10173E007405907FD4F07400907FD5F022907FEAEC
:10174E00E0FF123FA28B338A348935EA496011CE0D
:10175E00EACEEE907FD4F0CFE9CFEF907FD5F02296
:10176E00907FB4E04401F022907FEAE0FF1248003F
:10177E008B338A348935EA496011CEEACEEE907FFA
:10178E00D4F0CFE9CFEF907FD5F022907FB4E04434
:10179E0001F022907FEAE0FF907EC0E0FDA3E0FB27
:1017AE001244D28B338A348935EA496011CEEACE9F
:1017BE00EE907FD4F0CFE9CFEF907FD5F022907FDF
:1017CE00B4E04401F022907FB4E04401F022907F17
:0517DE00B4E04401F03D
:0117E30022E3
:1017E400C0E0C083C082907FC4E4F05391EF907F47
:0B17F400AB7404F0D082D083D0E03250
:0117FF0022C7
:10180000E4907815F07B0190781204F0A37478F0DE
:10181000A37458F0907812E0FBA3E0FAA3E0F990EB
:101820000001120C5DFF90799AE06F6018907815B6
:10183000E0C39406500FE004F0907813E475F00FC5
:10184000120CF480CF907815E0B40608907FB4E0D5
:101850004401F022907812E0FBA3E0FAA3E0F91231
:101860000C44FF24BF7002417A24E07002414C24F2
:101870002160024173907997E024FE7002219A144E
:10188000700221EF24026002414490792DE0A3F020
:10189000907923E0FFE4FCFDFEFBFA7901F8120DDC
:1018A00042C8ECC8C9EDC9CAEECACBEFCB907922C9
:1018B000E0FEE4FCFD2BFBEA3EFAED39F9EC38F8EA
:1018C000907921E0FFE4FEEB2FFFEE3AFEED39FDCB
:1018D000EC38FC907812E0FBA3E0FAA3E0F990006A
:1018E00002120DD2900002120DA27B447AAC790054
:1018F0007800C3120D91700590792D04F090781244
:10190000E0FBA3E0FAA3E0F9900002120DA27B80B5
:101910007ABB79007800C3120D91700690792D740E
:1019200002F0907812E0FBA3E0FAA3E0F990000245
:10193000120DA27B007A7779017800C3120D9170A5
:101940000690792D7403F090792DE0FFB4010975AC
:101950000C67750D06750E0BEFB40208E4F50CF577
:101960000D750E0CEFB40308E4F50CF50D750E18AB
:10197000EFB4030D90792EE064036005D22F123D81
:101980007990792DE06403600AA3E0B40305C22FC7
:10199000123D7912100012280122907923E0FFE411
:1019A000FCFDFEFBFA7901F8120D42C8ECC8C9ED46
:1019B000C9CAEECACBEFCB907922E0FEE4FCFD2B46
:1019C000FBEA3EFAED39F9EC38F8907921E0FFE4D2
:1019D000FEEB2FFFEE3AFEED39FDEC38FC9078126D
:1019E000E0FBA3E0FAA3E0F9900006120DD22290EA
:1019F0007923E0FFE4FCFDFEFBFA7901F8120D42C9
:101A0000C8ECC8C9EDC9CAEECACBEFCB907922E0C9
:101A1000FEE4FCFD2BFBEA3EFAED39F9EC38F890D8
:101A20007921E0FFE4FEEB2FFFEE3AFEED39FDEC0D
:101A300038FC907812E0FBA3E0FAA3E0F990000AEA
:101A4000120DD222907FB4E04401F022907997E009
:101A5000147018907921E0FF907812E0FBA3E0FA6F
:101A6000A3E0F990000EEF120C9C22907FB4E044AA
:0A1A700001F022907FB4E04401F081
:011A7A002249
:101A7B00E4FFFE7B0190780F04F0A37478F0A3745D
:101A8B002BF090780FE0FBA3E0FAA3E0F9900002B3
:101A9B00120C5DFD907FECE06D6013EFC39405506D
:101AAB000D0F907810E475F003120CF480D48D3385
:101ABB0090780FE0FBA3E0FAA3E0F9900001120C81
:101ACB005DFD907FEDE06D6013EEC3940B500D0E3A
:101ADB00907810E475F003120CF480D4907FEDE055
:101AEB00F534EF64056003BE0B08907FB4E044014E
:101AFB00F02290780FE0FBA3E0FAA3E0F9120C447C
:101B0B00FF24F06008240F700E12492A22124B8317
:0E1B1B00907920E534F022907FB4E04401F090
:011B29002299
:0F1B2A00907FEAE0B4FF04123416221238002232
:071B39005398FE5398FD32A2
:101B40000000000000000000000000000000000095
:101B50000000000000000000000000000000000085
:101B60000000000000000000000000000000000075
:101B70000000000000000000000000000000000065
:021F3E000000A1
:101F40000000000000000000000000000000000091
:101F50000000000000000000000000000000000081
:101F60000000000000000000000000000000000071
:101F70000000000000000000000000000000000061
:0527FC000000000022B6
:10280100907964E0146046147002413C2402600235
:10281100812A907FFC74CCF0907FFF74FCF090795A
:10282100787401F090797CE0907979F054FDF0446E
:1028310001F090797CF0A2AFE433F512C2AF120B34
:10284100A2E5126002D2AFE490797AF02290792D5C
:10285100E06401600201F1907FFC74CCF0907FFF95
:1028610074FCF09079787401F090797CE09079793A
:10287100F04401F04402F090797EE0B401099079CE
:1028810079E04404F08007907979E054FBF0907985
:1028910079E090797CF0A2AFE433F512C2AF120B6C
:1028A100A29079787402F0907984E0907979F0902F
:1028B100797FE0B40109907979E054FEF0800790C6
:1028C1007979E04401F0907979E054FDF054FBF01E
:1028D100907984F0120BA290797A7401F090796565
:1028E100F0E5126002D2AFE490798CF090798BF030
:1028F10090792DE0640260022196907FFC74C8F00B
:10290100907FFF74FCF09079787401F090797CE00D
:10291100907979F04401F04402F090797EE0B401BD
:1029210009907979E04404F08007907979E054FBCB
:10293100F0907979E090797CF0A2AFE433F512C29E
:10294100AF120BA29079787402F0907984E09079BB
:1029510079F090797FE0B40109907979E054FEF043
:102961008007907979E04401F0907979E04402F0B0
:1029710054FBF0907984F0120BA290797A7401F0F3
:102981009079657403F0E5126002D2AFE490798C1E
:10299100F090798BF090792DE064036002812A90A8
:1029A1007FFC7498F0907FFF74FCF090797874014B
:1029B100F090797CE0907979F04401F04402F09054
:1029C100797EE0B40109907979E04404F0800790C0
:1029D1007979E054FBF0907979E090797CF0A2AFBD
:1029E100E433F512C2AF120BA29079787402F09021
:1029F1007984E0907979F090797FE0B40109907958
:102A010079E054FEF08007907979E04401F0907903
:102A110079E054FDF04404F0907984F0120BA29017
:102A2100797A7401F09079657405F0E5126002D24B
:102A3100AFE490798CF090798BF02290792DE0645D
:102A410001600241E0907FFC74B4F0907FFF74FC60
:102A5100F09079787401F090797CE0907979F05474
:102A6100FEF04402F090797EE0B40109907979E0BA
:102A71004404F08007907979E054FBF0907979E093
:102A810090797CF0A2AFE433F512C2AF120BA290A1
:102A910079787402F0907984E0907979F090797F77
:102AA100E0B40109907979E054FEF08007907979DA
:102AB100E04401F0907979E054FDF054FBF0907915
:102AC10084F0120BA290797A7401F090796504F088
:102AD100E5126002D2AFE490798CF090798BF0909E
:102AE100792DE0640260026185907FFC74B0F09002
:102AF1007FFF74FCF09079787401F090797CE0901C
:102B01007979F054FEF04402F090797EE0B4010945
:102B1100907979E04404F08007907979E054FBF0F2
:102B2100907979E090797CF0A2AFE433F512C2AFED
:102B3100120BA29079787402F0907984E0907979FF
:102B4100F090797FE0B40109907979E054FEF0804A
:102B510007907979E04401F0907979E04402F054EA
:102B6100FBF0907984F0120BA290797A7401F090C5
:102B710079657404F0E5126002D2AFE490798CF0CB
:102B810090798BF090792DE064036002812A907F27
:102B9100FC7468F0907FFF74FCF09079787401F018
:102BA10090797CE0907979F054FEF04402F09079CC
:102BB1007EE0B40109907979E04404F080079079CE
:102BC10079E054FBF0907979E090797CF0A2AFE460
:102BD10033F512C2AF120BA29079787402F090799A
:102BE10084E0907979F090797FE0B4010990797966
:102BF100E054FEF08007907979E04401F090797912
:102C0100E054FDF04404F0907984F0120BA2907925
:102C11007A7401F09079657406F0E5126002D2AF22
:0A2C2100E490798CF090798BF0229A
:102C2B00E4FF7B0190781604F0A37478F0A374583A
:102C3B00F0907816E0FBA3E0FAA3E0F99000011204
:102C4B000C5DFE907FECE06E6013EFC39406500DAD
:102C5B000F907817E475F00F120CF480D4BF0608B0
:102C6B00907FB4E04401F022907816E0FBA3E0FAE9
:102C7B00A3E0F9120C44FF249F7002C1662421606B
:102C8B0002C18C907FE9E0247E7002A130147002A7
:102C9B00A1C824026002C15E900002120DA27B4407
:102CAB007AAC79007800C3120D917013907F007489
:102CBB0044F0A374ACF0E4A3F0907FB57403F090F0
:102CCB007816E0FBA3E0FAA3E0F9900002120DA244
:102CDB007B807ABB79007800C3120D917013907FC3
:102CEB00007480F0A374BBF0E4A3F0907FB5740381
:102CFB00F0907816E0FBA3E0FAA3E0F99000021243
:102D0B000DA27B007A7779017800C3120D916002D6
:102D1B00C193907F00F0A37477F0A37401F0907FC0
:102D2B00B57403F022907816E0FBA3E0FAA3E0F968
:102D3B00900006120DA27B447AAC79007800C31286
:102D4B000D917013907F007444F0A374ACF0E4A366
:102D5B00F0907FB57403F0907816E0FBA3E0FAA334
:102D6B00E0F9900006120DA27B807ABB7900780007
:102D7B00C3120D917013907F007480F0A374BBF09D
:102D8B00E4A3F0907FB57403F0907816E0FBA3E01A
:102D9B00FAA3E0F9900006120DA27B007A77790175
:102DAB007800C3120D916002C193907F00F0A37461
:102DBB0077F0A37401F0907FB57403F0229078162E
:102DCB00E0FBA3E0FAA3E0F990000A120DA27B440A
:102DDB007AAC79007800C3120D917013907F007458
:102DEB0044F0A374ACF0E4A3F0907FB57403F090BF
:102DFB007816E0FBA3E0FAA3E0F990000A120DA20B
:102E0B007B807ABB79007800C3120D917013907F91
:102E1B00007480F0A374BBF0E4A3F0907FB574034F
:102E2B00F0907816E0FBA3E0FAA3E0F990000A1209
:102E3B000DA27B007A7779017800C3120D9170484F
:102E4B00907F00F0A37477F0A37401F0907FB574BA
:102E5B0003F022907FB4E04401F022907FE9E0245C
:102E6B007F7016907816E0FBA3E0FAA3E0F99000D0
:102E7B000E120C5D907F00F022907FB4E04401F0C5
:082E8B0022907FB4E04401F045
:012E9300221C
:102E9400753625753724907974E064017054F0F523
:102EA40035752201E52264017048907FA5E04480D5
:102EB400F0907FA6E536F01246C0744F2535F582B2
:102EC400E43479F583E0907FA6F01246C07435258A
:102ED40035F582E43479F583E0907FA6F01246C09C
:102EE400907FA57440F0120ACD0535E535C3940DE5
:102EF40040B2907975E064016002E1DEF0907920DF
:102F0400E064056002E18D7B0190795C04F0A374B8
:102F140078F0A374B2F075330790795CE0FBA3E01A
:102F2400FAA3E0F9900001120C5D700F90000412F6
:102F34000C5D90792FF0120C29800690792F74FF84
:102F4400F0E4F535752201753402E5226401703927
:102F5400907FA5E04480F0907FA6E536F01246C04D
:102F6400AF340534907FA6EFF01246C090792FE07D
:102F7400907FA6F01246C0907FA57440F0120ACD4F
:102F84000535E535C3940640C1907920E0640670A8
:102F9400497B0190795F04F0A37478F0A374FFF087
:102FA40075330390795FE0FBA3E0FAA3E0F99000A6
:102FB40001120C5D701C900004120C5D907933F0CA
:102FC400700374FFF0907933E0547FFFF025E0F054
:0A2FD4008005E4907933F01247DF26
:012FDE0022D0
:102FDF009079787403F0907983E0907979F0A2AFCB
:102FEF00E433F512C2AF120BA2E5126002D2AF2288
:012FFF0022AF
:10300000E4FE907920E0FDB405119078257401F07C
:10301000A37478F0A374B2F0753507EDB40611907F
:1030200078257401F0A37478F0A374FFF07535036C
:10303000907FEBE014601114605B24026002410594
:10304000907FB4E04401F022907FE9E0247F703D5E
:10305000E4FFEFC39535502F907825E0FBA3E0FA0D
:10306000A3E0F9900001120C5DFDCCEECC0E7400D3
:103070002CF582E4347FF583EDF0907826E475F04A
:103080000B120CF40F80CB907FB5EEF022907FB442
:10309000E04401F022907FE9E0247E606414700235
:1030A000215514700221A92403600221FDE4FFEFE1
:1030B000C395355046907825E0FBA3E0FAA3E0F9EC
:1030C000900003120C5DFDCCEECC0E74002CF5824A
:1030D000E4347FF583EDF0900004120C5DFDCCEE3E
:1030E000CC0E74002CF582E4347FF583EDF09078FB
:1030F00026E475F00B120CF40F80B4907FB5EEF05F
:1031000022E4FFEFC395355046907825E0FBA3E01D
:10311000FAA3E0F9900005120C5DFDCCEECC0E7424
:10312000002CF582E4347FF583EDF0900006120C5C
:103130005DFDCCEECC0E74002CF582E4347FF5837B
:10314000EDF0907826E475F00B120CF40F80B4903B
:103150007FB5EEF022E4FFEFC39535504690782519
:10316000E0FBA3E0FAA3E0F9900007120C5DFDCCB0
:10317000EECC0E74002CF582E4347FF583EDF090F4
:103180000008120C5DFDCCEECC0E74002CF582E430
:10319000347FF583EDF0907826E475F00B120CF493
:1031A0000F80B4907FB5EEF022E4FFEFC395355069
:1031B00046907825E0FBA3E0FAA3E0F9900009121D
:1031C0000C5DFDCCEECC0E74002CF582E4347FF562
:1031D00083EDF090000A120C5DFDCCEECC0E740075
:1031E0002CF582E4347FF583EDF0907826E475F0D9
:1031F0000B120CF40F80B4907FB5EEF022907FB4E8
:0C320000E04401F022907FB4E04401F0B3
:01320C00229F
:10320D007B017A78792B907800EBF0A3EAF0A3E9B3
:10321D00F07401120C8A907800E0FBA3E0FAA3E0B1
:10322D00F99000017401120C9C900002E4120C9CA8
:10323D00907801E475F003120CF4907800E0FBA394
:10324D00E0FAA3E0F97410120C8A907800E0FBA369
:10325D00E0FAA3E0F99000017405120C9C900002B5
:10326D00E4120C9C907801E475F003120CF4907844
:10327D0000E0FBA3E0FAA3E0F97402120C8A907847
:10328D0000E0FBA3E0FAA3E0F99000017402120C38
:10329D009C900002E4120C9C907801E475F00312EE
:1032AD000CF4907800E0FBA3E0FAA3E0F9740112AE
:1032BD000C8A907800E0FBA3E0FAA3E0F9900001FE
:1032CD007403120C9C900002E4120C9C907801E4A3
:1032DD0075F003120CF4907800E0FBA3E0FAA3E084
:1032ED00F97410120C8A907800E0FBA3E0FAA3E0C9
:1032FD00F99000017406120C9C900002E4120C9CD3
:10330D00907801E475F003120CF4907800E0FBA3C3
:10331D00E0FAA3E0F97402120C8A907800E0FBA3A6
:10332D00E0FAA3E0F99000017404120C9C900002E5
:10333D00E4120C9C907801E475F003120CF4907873
:10334D0000E0FBA3E0FAA3E0F97402120C8A907876
:10335D0000E0FBA3E0FAA3E0F99000017404120C65
:10336D009C9000027404120C9C907801E475F0039B
:10337D00120CF4907800E0FBA3E0FAA3E0F97402DC
:10338D00120C8A907800E0FBA3E0FAA3E0F990001C
:10339D00017403120C9C9000027404120C9C907822
:1033AD0001E475F003120CF4907800E0FBA3E0FA51
:1033BD00A3E0F97402120C8A907800E0FBA3E0FA06
:1033CD00A3E0F99000017402120C9C9000027404A9
:1033DD00120C9C907801E475F003120CF4907800B7
:1033ED00E0FBA3E0FAA3E0F97402120C8A907800D6
:1033FD00E0FBA3E0FAA3E0F99000017401120C9C2C
:08340D009000027404120C9CF3
:013415002294
:10341600E4FE907920E0FDB4051190781F7401F068
:10342600A37478F0A374B2F0753507EDB406119065
:10343600781F7401F0A37478F0A374FFF075350358
:10344600907999E014601114605B24026002C10651
:10345600907FB4E04401F022907997E014703EE446
:10346600FFEFC39535502FCDEECD0E74212DF5828D
:10347600E43479F583E0FD90781FE0FBA3E0FAA33E
:10348600E0F9900001ED120C9C907820E475F00BA9
:10349600120CF40F80CB9079757401F022907FB4F2
:1034A600E04401F022907997E024FE6063147002F4
:1034B600A164147002A1B224036002A1FEE4FFEF2E
:1034C600C395355044CDEECD0E74212DF582E434EE
:1034D60079F583E0FD90781FE0FBA3E0FAA3E0F91D
:1034E600900003ED120C9CCDEECD0E74212DF582CD
:1034F600E43479F583E0900004120C9C907820E483
:1035060075F00B120CF40F80B69079757401F022E9
:10351600E4FFEFC395354002C10DCDEECD0E74210B
:103526002DF582E43479F583E0FD90781FE0FBA366
:10353600E0FAA3E0F9900005ED120C9CCDEECD0E5D
:1035460074212DF582E43479F583E0900006120C9F
:103556009C907820E475F00B120CF40F80B4E4FF15
:10356600EFC395354002C10DCDEECD0E74212DF57C
:1035760082E43479F583E0FD90781FE0FBA3E0FA5E
:10358600A3E0F9900007ED120C9CCDEECD0E742150
:103596002DF582E43479F583E0900008120C9C90B6
:1035A6007820E475F00B120CF40F80B4E4FFEFC33F
:1035B60095355053CDEECD0E74212DF582E4347938
:1035C600F583E0FD90781FE0FBA3E0FAA3E0F99015
:1035D6000009ED120C9CCDEECD0E74212DF582E482
:1035E6003479F583E090000A120C9C907820E475FB
:1035F600F00B120CF40F80B6907FB4E04401F02279
:07360600907FB4E04401F0E5
:01360D00229A
:10360E00E4FE907920E0FDB405109078287401F066
:10361E00A37478F0A374B2F07F07EDB4061090781F
:10362E00287401F0A37478F0A374FFF07F039078F0
:10363E0028E0FBA3E0FAA3E0F9120C44FD907FEA28
:10364E00E06D6012EEC39F500D907829E475F00B7B
:10365E00120CF40E80D8907FEBE0146011146046CB
:10366E0024026002E19A907FB4E04401F022907F40
:10367E00E9E0247F7028EE6F7008907FB4E044017B
:10368E00F022907828E0FBA3E0FAA3E0F990000185
:10369E00120C5D907F00F0907FB57401F022907F48
:1036AE00B4E04401F022907FE9E0247E6040146093
:1036BE006F147002E16024036002E192EE6F7008F5
:1036CE00907FB4E04401F022907828E0FBA3E0FA6A
:1036DE00A3E0F9900003120C5D907F00F0900004BF
:1036EE00120C5D907F01F0907FB57402F022EE6FA8
:1036FE007008907FB4E04401F022907828E0FBA39C
:10370E00E0FAA3E0F9900005120C5D907F00F090B6
:10371E000006120C5D907F01F0907FB57402F022CE
:10372E00EE6F7008907FB4E04401F022907828E0AC
:10373E00FBA3E0FAA3E0F9900007120C5D907F0066
:10374E00F0900008120C5D907F01F0907FB574022E
:10375E00F022EE6F7008907FB4E04401F022907872
:10376E0028E0FBA3E0FAA3E0F9900009120C5D90AB
:10377E007F00F090000A120C5D907F01F0907FB5F3
:10378E007402F022907FB4E04401F022907FB4E006
:03379E004401F0F3
:0137A1002205
:1037A200C0E0C0F0C083C082C0D0E8C0E0E9C0E0A1
:1037B200EAC0E0EBC0E0ECC0E0EDC0E0EEC0E0EF5C
:1037C200C0E05391EF907FAB7410F0907983E05496
:1037D200FDF0122FDFD0E0FFD0E0FED0E0FDD0E020
:1037E200FCD0E0FBD0E0FAD0E0F9D0E0F8D0D0D0C5
:0837F20082D083D0F0D0E03258
:0637FA005391BFD22632FC
:10380000E4FE907920E0FDB405109078227401F078
:10381000A37478F0A374B2F07F07EDB4061090782B
:10382000227401F0A37478F0A374FFF07F03907802
:1038300022E0FBA3E0FAA3E0F9120C44FD90799892
:10384000E06D6012EEC39F500D907823E475F00B8D
:10385000120CF40E80D8907999E01460111460482D
:10386000240260022185907FB4E04401F022907927
:1038700097E014702BEE6F7009907FB4E04401F074
:103880008017907921E0FD907822E0FBA3E0FAA375
:10389000E0F9900001ED120C9C9079757401F02212
:1038A000907FB4E04401F022907997E024FE6043D9
:1038B00014606E147002214F24036002217DEE6FAC
:1038C0007009907FB4E04401F08021907921E0FDFF
:1038D000907822E0FBA3E0FAA3E0F9900003ED1258
:1038E0000C9C907922E0900004120C9C90797574E5
:1038F00001F022EE6F7008907FB4E04401F0229056
:103900007921E0FD907822E0FBA3E0FAA3E0F990B2
:103910000005ED120C9C907922E0900006120C9CA0
:1039200022EE6F7008907FB4E04401F0229079217C
:10393000E0FD907822E0FBA3E0FAA3E0F990000715
:10394000ED120C9C907922E0900008120C9C22EE63
:103950006F7008907FB4E04401F022907921E0FE7E
:10396000907822E0FBA3E0FAA3E0F9900009EE12C0
:103970000C9C907922E090000A120C9C22907FB45B
:0C398000E04401F022907FB4E04401F02C
:01398C002218
:10398D00A2AFE433F512E4907983F0122FDF907F2C
:10399D00E07490F0907FE17404F0E4907FDDF0909E
:1039AD007FA1F0538EF875880575B82075F8014321
:1039BD008E30F5C875CA7F75CBF843A82090797401
:1039CD0004F0C222E4F50F907978F0A3F0907962BB
:1039DD00F0A3F0A3F0907966F0A3F090797BF0A3BB
:1039ED00F0907984F090797DF0907975F0A3F0A343
:1039FD00F0C223C224C225C226C220907F9BE0F5CF
:103A0D000A5420F50A700690797EF0800690797E32
:103A1D007401F0907F9BE0F50A5402F50A70069050
:103A2D00797FF0800690797F7401F0907978740237
:103A3D00F0907984E0907979F090797FE0B4010984
:103A4D00907979E054FEF08007907979E04401F0A7
:103A5D00907979E0907984F0120BA29079787401C5
:103A6D00F090797CE0907979F090797EE0B401095D
:103A7D00907979E04404F08007907979E054FBF077
:103A8D00907979E090797CF0120BA2E4907978F03E
:103A9D00A304F0E4907988F0120BA2907FFC74DD02
:103AAD00F0907FFF74FFF09079787401F0A3F0121D
:103ABD000BA2E490797AF090798304F0122FDFE471
:103ACD00907930F0907985F0A3F0A3F0122E9490B8
:103ADD00792D7402F090798814F0C22FE4907968F2
:103AED00F090798AF090796AF0A3F0751308751447
:103AFD0008F516F515F51790798CF090798BF02265
:103B0D007B017A787958907803EBF0A3EAF0A3E97A
:103B1D00F07440120C8A907803E0FBA3E0FAA3E066
:103B2D00F9900001740A120C9C900002120DF6001F
:103B3D0000BB80900006120DF60000AC4490000A08
:103B4D00120DF600017700907804E475F00F120C59
:103B5D00F4907803E0FBA3E0FAA3E0F97440120CB3
:103B6D008A907803E0FBA3E0FAA3E0F990000174DA
:103B7D008C120C9C900002120DF60000BB80900080
:103B8D0006120DF60000AC4490000A120DF600016D
:103B9D007700907804E475F00F120CF4907803E040
:103BAD00FBA3E0FAA3E0F97440120C8A907803E0CD
:103BBD00FBA3E0FAA3E0F9900001748F120C9C9026
:103BCD007804E475F00F120CF4907803E0FBA3E099
:103BDD00FAA3E0F97441120C8A907803E0FBA3E09C
:103BED00FAA3E0F99000017484120C9C907804E41F
:103BFD0075F00F120CF4907803E0FBA3E0FAA3E04C
:103C0D00F97461120C8A907803E0FBA3E0FAA3E04B
:103C1D00F99000017481120C9C907804E475F00FFA
:103C2D00120CF4907803E0FBA3E0FAA3E0F97461C1
:103C3D00120C8A907803E0FBA3E0FAA3E0F9900060
:063C4D00017401120C9C41
:013C5300224E
:103C5400C0E0C0F0C083C082C0D0E8C0E0E9C0E0EA
:103C6400EAC0E0EBC0E0ECC0E0EDC0E0EEC0E0EFA5
:023C7400C0E0AE
:103C7600907FA2E0F50B907F74E0907970F0907FD2
:103C860075E0907971F0907983E0FFFE5402FE7042
:103C96000DEF4402F0122FDF9079747401F0E50BFA
:103CA60020E228907970E0FEA3E07C002400F51164
:103CB600EC3EF510907982E0FDAE10AF11120CBE0D
:103CC600907970EFF09079897401F01248431248A8
:103CD60076907989E064017032124108907989E41E
:103CE600F0907F98E04440F0907F9EE04440F09052
:103CF6007F957480F075E80112093275E80D907FA2
:103D06009574C0F075E80DD220800575E801C220D3
:103D160020202B90792DE0FFB40109750C67750DF5
:103D260006750E0BEFB40209750C00750D00750EC5
:103D36000CEFB40309750C00750D00750E1875CAE5
:103D46006F75CBFED2CA5391EF907FAB7402F0F041
:103D5600D0E0FFD0E0FED0E0FDD0E0FCD0E0FBD02C
:103D6600E0FAD0E0F9D0E0F8D0D0D082D083D0F01D
:033D7600D0E03268
:103D790075332575342490795C7401F0A37478F057
:103D8900A374B2F0202F02C117E4F5357522019012
:103D9900795CE0FBA3E0FAA3E0F9900004120C5D62
:103DA900F53675350674422535F582E43479F5839F
:103DB900E536F00535E535B40CEBE535C3940D4032
:103DC90002C198E52264016002C198907FA5E04490
:103DD90080F0907FA6E533F01246C0744F2535F583
:103DE90082E43479F583E0907FA6F01246C07442EC
:103DF9002535F582E43479F583E0907FA6F0124603
:103E0900C0907FA57440F0120ACD053580ACE4F569
:103E19003575220190795CE0FBA3E0FAA3E0F99003
:103E29000004120C5DF53675350674352535F582B5
:103E3900E43479F583E536F00535E535B40CEBE581
:103E490035C3940D5049E52264017043907FA5E084
:103E59004480F0907FA6E533F01246C0744F2535B3
:103E6900F582E43479F583E0907FA6F01246C074B8
:103E7900352535F582E43479F583E0907FA6F01293
:0F3E890046C0907FA57440F0120ACD053580B079
:013E98002207
:103E99009078097401F0A37478F0A374B2F0E4FF88
:103EA900FE907809E0FBA3E0FAA3E0F9EF120C8A8F
:103EB900907809E0FBA3E0FAA3E0F9900001E4128D
:103EC9000C9C9000027415120C9C900003E4120CD7
:103ED9009C90000474FF120C9C900005E4120C9C49
:103EE90090000674C3120C9C900007E4120C9C907D
:103EF9000008E4120C9C900009E4120C9C90000A42
:103F09007401120C9C90780AE475F00B120CF40FF2
:103F19000EBE078D9078097401F0A37478F0A3742C
:103F2900FFF0E4FFFE907809E0FBA3E0FAA3E0F9D3
:103F3900EF120C8A907809E0FBA3E0FAA3E0F9906C
:103F49000001E4120C9C9000027415120C9C900064
:103F590003E4120C9C9000047480120C9C900005E0
:103F6900E4120C9C90000674C3120C9C900007E4A8
:103F7900120C9C900008E4120C9C900009E4120CAD
:103F89009C90000A7401120C9C90780AE475F00B5D
:083F9900120CF40F0EBE038DA3
:013FA10022FD
:103FA200E4FE753DFF753E05753F12AB3DAA3EA985
:103FB2003F900001120C5D6402702FCDEECD0EED2C
:103FC2006F700122900002120D0A85F03BF53C62EF
:103FD2003BE53B623CE53C623B29FDE53B3AC9EDF2
:103FE200C9753DFFF53E893F80C17B007A007900AB
:013FF20022AC
:093FF30053D8EF43D820C22D324F
:043FFC005391DF32CC
:10400000907987E0B4011D907985E0B401031242F4
:10401000AA907986E0B40103121800E4907985F043
:10402000A3F0A3F0122E94907F9BE0F50A5402F5C2
:104030000A700490797FF0907F9BE0F50A5402FFAC
:10404000F50ABF020690797F7401F0907F9BE0F53E
:104050000A5420F50A700490797EF0907F9BE0F579
:104060000A5420FFF50ABF200690797E7401F09073
:10407000797FE0FF907981E06F6038907978740201
:10408000F0907984E0907979F0EFB40106E054FE85
:10409000F08007907979E04401F0907979E09079A7
:1040A00084F0A2AFE433F512C2AF120BA2E51260A6
:1040B00002D2AF90797EE0FF907980E06F60389017
:1040C00079787401F090797CE0907979F0EFB4011F
:1040D00006E04404F08007907979E054FBF0907991
:1040E00079E090797CF0A2AFE433F512C2AF120B05
:1040F000A2E5126002D2AF90797FE0907981F090D2
:08410000797EE0907980F02245
:1041080090792DE064017035907970E0FFD3942D9B
:10411800402B9079697401F0907968E004F0E0D35D
:10412800940F4019E4F0EFD39431400890792D743E
:1041380003F0800690792D7402F012100090792D0A
:10414800E0B4022C907970E0FFC3942F5022EFD393
:10415800942A401C9079697401F0907968E004F021
:10416800E0D3940F400AE4F090792D04F012100087
:1041780090792DE0B40226907970E0D39431401DF7
:104188009079697401F0907968E004F0E0D3940FB5
:10419800400BE4F090792D7403F012100090792D03
:1041A800E06403703F907970E0FFC3945F503590EE
:1041B80079697401F0907968E004F0E0D3940F40D5
:1041C80023E4F0EFC3942F500CEFD3942A400690C9
:1041D800792D7401F0EFD3942F400690792D740255
:1041E800F0121000907969E07005907968F022E487
:0541F800907969F0223E
:1041FD007B017A78794C907806EBF0A3EAF0A3E98D
:10420D00F0E4120C8A907806E0FBA3E0FAA3E0F943
:10421D009000017401120C9C907807E475F0031264
:10422D000CF4907806E0FBA3E0FAA3E0F9E4120C9D
:10423D008A907806E0FBA3E0FAA3E0F99000017400
:10424D0002120C9C907807E475F003120CF4907830
:10425D0006E0FBA3E0FAA3E0F9E4120C8A907806DD
:10426D00E0FBA3E0FAA3E0F99000017403120C9CAB
:10427D00907807E475F003120CF4907806E0FBA338
:10428D00E0FAA3E0F9E4120C8A907806E0FBA3E0D3
:0C429D00FAA3E0F99000017404120C9CDC
:0142A90022F2
:1042AA00E4FFFE7B0190780C04F0A37478F0A37409
:1042BA002BF090780CE0FBA3E0FAA3E0F99000025F
:1042CA00120C5DFD90799AE06D6013EFC39405506E
:1042DA000D0F90780DE475F003120CF480D48D3331
:1042EA0090780CE0FBA3E0FAA3E0F9900001120C2D
:1042FA005DFD90799BE0FC6D6013EEC3940B500D4D
:10430A000E90780DE475F003120CF480D38C34EF20
:10431A0064056003BE0B08907FB4E04401F022906C
:10432A00780CE0FBA3E0FAA3E0F9120C44FF24F0B6
:10433A006008240E700E12494D22907920E534F05F
:0B434A00121B2A22907FB4E04401F017
:014355002245
:0C435600787FE4F6D8FD75813F02439D9E
:104362000248A9E493A3F8E493A34003F68001F280
:1043720008DFF48029E493A3F85407240CC8C3335C
:10438200C4540F4420C8834004F456800146F6DF2B
:10439200E4800B0102040810204080904661E47E14
:1043A200019360BCA3FF543F30E509541FFEE49320
:1043B200A360010ECF54C025E060A840B8E493A3E7
:1043C200FAE493A3F8E493A3C8C582C8CAC583CA12
:1043D200F0A3C8C582C8CAC583CADFE9DEE780BECA
:1043E200C0E0C0F0C083C082C0D0E8C0E0E9C0E055
:1043F200EAC0E0EBC0E0ECC0E0EDC0E0EEC0E0EF10
:10440200C0E0C2CAC2CF90797AE0B4011F124BAEAB
:1044120012475853A8A0907FAEE4F01207AA124B9D
:10442200B7907FAE741FF043A805800353A8A05332
:10443200A8FA75E80112091575E80D43A805D0E040
:10444200FFD0E0FED0E0FDD0E0FCD0E0FBD0E0FA0F
:10445200D0E0F9D0E0F8D0D0D082D083D0F0D0E054
:014462003227
:10446300907FECE0F50914601D14602A1460371482
:10447300604424047050907962E0907F00F0907F54
:10448300B57401F08047907963E0907F00F0907FEE
:10449300B57401F08037907964E0907F00F0907FED
:1044A300B57401F08027907966E0907F00F0907FEB
:1044B300B57401F08017907967E0907F00F0907FEA
:0F44C300B57401F08007907FB4E04401F0D3227C
:0444D2008D368B3761
:1044D600123FA2EA496057120C447E0029FFEE3AC9
:1044E600C9EFC97538FFF539893AAB38AA39A93AFF
:1044F600900001120C5DFF64046005EF6405702EE8
:10450600EFB40415900002120C5D6536700B900036
:1045160003120C5D6537700122120C447E0029FFE0
:10452600EE3AC9EFC97538FFF539893A80BC7B0088
:044536007A0079008E
:01453A00225E
:10453B00E4FF7B0190781C04F0A37478F0A3744C17
:10454B00F090781CE0FBA3E0FAA3E0F990000212D4
:10455B000C5DFE907FECE06E6013EFC39404500D86
:10456B0090781DE475F003120CF40F80D4BF04098E
:10457B00907FB4E04401F08014907921E0FF9078B3
:10458B001CE0FBA3E0FAA3E0F9EF120C8A907FC5C5
:03459B007401F0B8
:01459E0022FA
:0E459F00C0E0C083C082C0D0EEC0E0EFC0E03C
:1045AD00907985E064016005A3E0B4012D907987D1
:1045BD007401F0E4FF907FC5E0FEEFC39E501B74C5
:1045CD00C02FF582E4347EF583E0FE74212FF58251
:1045DD00E43479F583EEF00F80DB5391EF907FAAF1
:0445ED00E04401F0B5
:0F45F100D0E0FFD0E0FED0D0D082D083D0E03237
:10460000E4FF7B0190781904F0A37478F0A3744C54
:10461000F0907819E0FBA3E0FAA3E0F99000021211
:104620000C5DFE907FECE06E6013EFC39404500DC0
:1046300090781AE475F003120CF40F80D4BF0408CC
:10464000907FB4E04401F022907819E0FBA3E0FAF7
:10465000A3E0F9120C44907F00F0907FB57401F054
:014660002237
:1046610001180201190A011C00C128C129011F01F9
:0F46710044799F000000004179A3004179A40023
:0446800041798900F3
:10468400012201417931FF417934004D79353F3FB1
:1046940000080001000000000000154D79423F3F72
:1046A40006080407000000000000154D794F0A0AAF
:0B46B4000900010902030405060708C5
:0146BF0000FA
:1046C000120ACD907FA5E0F521E5215401F5216482
:1046D000016028E52264017022907FA5E0F5215455
:1046E00002F5217003752201907FA5E0F5215404A5
:0C46F000FFF521BF04D375220180CE220B
:0446FC0053D8F73266
:104700000249FA00023C54000217E400024A120077
:104710000237A2000247FF00024A410002459F0003
:1047200002498E000249AB00024A5800024A6F005B
:10473000024A8600024A9D00024AB400024ACB00A7
:10474000024AE200024AF900024B1000024B270025
:08475000024B3E00024B550034
:10475800E518701490798CE004F090798BE0C3949C
:10476800004015E014F0801090798BE004F0A3E08D
:10477800C394004003E014F090798BE0D394144084
:1047880004E4F518F090798CE0D39414400575187A
:0447980001E4F02226
:10479C00907FD7E0F533907FECE0F50914601114AD
:1047AC00601B24027024907FEAE0907962F08021F3
:1047BC00907FEAE0907963F01210008014907FEA09
:1047CC00E0907964F01228018007907FB4E04401F6
:0247DC00F0D318
:0147DE0022B8
:1047DF009079787404F0907933E0907979F0A2AF02
:1047EF00E433F512C2AF120BA2E5126002D2AF2270
:0147FF003287
:024800008F36F1
:10480200E4F5377538FF753907753A01AB38AA39BF
:10481200A93A900001120C5DB4031FAF370537EFC0
:104822006536700122120C447E0029FFEE3AC9EF70
:10483200C97538FFF539893A80D27B007A00790050
:014842002253
:1048430030262FC22690792DE0FFB40109E4F50C40
:10485300750DF8750E0AEFB40209E4F50C750DF049
:10486300750E0BEFB40309E4F50C750DF8750E170F
:03487300D222222C
:1048760030252FC22590792DE0FFB40109750CC0B3
:10488600750D14750E0BEFB40209E4F50C750D10D9
:10489600750E0CEFB40309E4F50C750D18750E18BA
:0348A600D22222F9
:1048A900E4F532120F50202E10E532C3940250095C
:1048B9000532D23012490580ED302E05121457C247
:0F48C9002E302D0612079A1248D912400080EAAD
:0148D80022BD
:1048D900907FD6E0F51D5480F51D6480701DC2AF30
:1048E900E04480F0E04401F07F0C7E00124B6C90B4
:0C48F9007FD6E054FEF05387FED2AF22C1
:10490500907FD6E054FBF0E04408F0303004E044FA
:1049150002F07FDC7E05124B6C907FD6E054F7F0F9
:05492500E04404F02253
:10492A00907FEBE0147014907FE9E0247F7004120A
:10493A00460022907FB4E04401F022907FB4E04424
:03494A0001F02257
:10494D00907FEBE0147013907FE9E0147004124532
:10495D003B22907FB4E04401F022907FB4E044010B
:02496D00F02236
:10496F00E4FF74E82FF582E4347FF583E0FE74965C
:0E497F002FF582E43479F583EEF00FBF08E4E3
:01498D002207
:10498E00C0E0C083C0825391EF907FA9E04402F053
:0D499E00907FB77403F0D082D083D0E03258
:1049AB00C0E0C083C0825391EF907FAAE04402F035
:0D49BB00907FC77403F0D082D083D0E0322B
:1049C800907FD6E030E712E04401F07F147E0012B9
:0A49D8004B6C907FD6E054FEF022F5
:1049E200E4F51A751B0190799104F0A3F0E4A3F0A9
:0849F200A3740AF0E4A3F02213
:1049FA00C0E0C083C082D22E5391EF907FAB740186
:084A0A00F0D082D083D0E0322D
:104A1200C0E0C083C082D22D5391EF907FAB740867
:084A2200F0D082D083D0E03215
:104A2A00907FEAE0F508E4907962F0A3F0A3F090B1
:074A3A007966F0A3F0D3221E
:104A4100C0E0C083C0825391EF907FA9E04401F0A0
:074A5100D082D083D0E032D7
:104A5800C0E0C083C0825391EF907FA9E04404F086
:074A6800D082D083D0E032C0
:104A6F00C0E0C083C0825391EF907FAAE04404F06E
:074A7F00D082D083D0E032A9
:104A8600C0E0C083C0825391EF907FA9E04408F054
:074A9600D082D083D0E03292
:104A9D00C0E0C083C0825391EF907FAAE04408F03C
:074AAD00D082D083D0E0327B
:104AB400C0E0C083C0825391EF907FA9E04410F01E
:074AC400D082D083D0E03264
:104ACB00C0E0C083C0825391EF907FAAE04410F006
:074ADB00D082D083D0E0324D
:104AE200C0E0C083C0825391EF907FA9E04420F0E0
:074AF200D082D083D0E03236
:104AF900C0E0C083C0825391EF907FAAE04420F0C8
:074B0900D082D083D0E0321E
:104B1000C0E0C083C0825391EF907FA9E04440F091
:074B2000D082D083D0E03207
:104B2700C0E0C083C0825391EF907FAAE04440F079
:074B3700D082D083D0E032F0
:104B3E00C0E0C083C0825391EF907FA9E04480F023
:074B4E00D082D083D0E032D9
:104B5500C0E0C083C0825391EF907FAAE04480F00B
:074B6500D082D083D0E032C2
:104B6C008E338F34E5341534AE33700215334E600A
:074B7C000512078980EE22FB
:0F4B8300907FEAE0B4FF041230002212360E22B7
:0E4B9200C0E0C28BD224302302C223D0E03216
:0E4BA000907F00E508F0907FB57401F0D322FD
:094BAE00302405C224751801220F
:094BB700302305C223E4F51822A5
:074BC00053C0FE53C0FD329B
:064BC70053917FD225325C
:054BCD00C289D2233271
:034BD200C28D325F
:034BD500C28F325A
:024BD800D322E6
:024BDA00D322E4
:024BDC00D322E2
:024BDE00D322E0
:024BE000D322DE
:024BE200D322DC
:024BE400C322EA
:014BE60022AC
:00000001FF
